:020000003628A0
:080008008C00030E8D00830142
:100010000B1910280B1817280B08F8398B003028FB
:100020000B118F0B2328900A40308F0023281718BC
:100030000530971804301719033097190230171A32
:100040000830980030289708031D980B302828287E
:10005000191C2D2886101910172886141914172812
:100060000B100D0E83008C0E0C0E090083169830B9
:100070008100FF30850083129401970199013C3083
:100080008600051C9914851C19150030051D0230C9
:10009000831686008312103096001630051E083035
:1000A0009607030191018421030191018421030139
:1000B0009101842103019101842103019101842193
:1000C000030191018421030191018421A8308B0057
:1000D00001089A0086010301910184210301910125
:1000E0008421140C031C78281608103C031C96036A
:1000F000010899181A0892002521940A0A219501ED
:10010000950A140819199500403C0319FA28AA30D9
:100110009100030184211D211230840038217921AE
:10012000191998281408150203189A28950A87287F
:10013000950B872899186B289501950A14081919A9
:1001400095001D2140308F0090014A219300063018
:1001500091000301842113308400382140308F0046
:1001600090010B145721860197010630910003017D
:10017000842112081302031DC8281919C528140860
:10018000150203186B28950AA128950BA1286B2846
:1001900086011230840038214030960097011716EE
:1001A00079210301910184210301910184219501A9
:1001B0000A301402031CDF28950A9400D8289508F9
:1001C0000319EC28203096009701171479210301B8
:1001D00091018421950BDF289408031963001030E6
:1001E0009600970197157921030191018421940BC1
:1001F000EC28630007309600053091009701171432
:100200007921971479211715792197157921910B67
:10021000FF286300140889001208880083168B13D6
:10022000081555308900AA30890088148B170811E9
:10023000081E182908128312080015088900831661
:10024000081483120808920008000310920D120E81
:10025000E039920C120712071207353C92009A00FF
:10026000920D8E018E0D920D8E0D0E0892000800DB
:100270008018422900183F29061517140800861512
:100280009714080000184729061617150800861647
:1002900097150800051C0034851C0134051D023427
:1002A000851D03341008C83C0319C8284A2993182F
:1002B000692913186229051808001008C83C031999
:1002C000C8285B29851808001008C83C0319C828ED
:1002D000622913187229051908001008C83C03196F
:1002E000C8286B29851908001008C83C0319C828BC
:1002F000722940308F0090010B1416081002031D64
:100300007D29860197010800013E031D8429910B78
:040310008429080034
:02400E00F33F7E
:00000001FF
